:100000008A01830102290000FF00030EFE0004089C
:10001000FC000A08FD008A01830183120C1C1528CC
:1000200018308A00E12883120C1083128B1C1D28C3
:1000300018308A00012883128B107D088A007C0802
:1000400084007E0E8300FF0E7F0E090008308A00B8
:10005000012817308A002A2F16308A00D62E083041
:100060008A006B280A308A009C2A0A308A00B92A42
:100070000A308A00B92A0A308A00F22A09308A0036
:100080004F2909308A00FD2908308A009528093057
:100090008A002F290B308A00222B0B308A00782B04
:1000A0000B308A00942B0A308A00282A0A308A00F2
:1000B0007A2A0A308A00922A10308A0001281030E9
:1000C0008A00112812308A00F42A12308A00FE2A8F
:1000D00013308A009D2B13308A00792B13308A004D
:1000E0008B2B13308A00432B13308A00552B13308F
:1000F0008A00672B13308A00B32B13308A00DB2B66
:1001000014308A00032C14308A00372C14308A00F3
:100110006B2C14308A00B72C15308A00032D153053
:100120008A00372D15308A006B2D15308A009F2DDF
:1001300016308A00072E16308A00152E15308A00D8
:10014000D32D16308A00232E16308A003D2E16300D
:100150008A002F2E12308A002B2A12308A00F62AAB
:1001600013308A009F2B13308A007B2B13308A00B8
:100170008D2B13308A00452B13308A00572B1330F8
:100180008A00692B13308A00C12B13308A00E92BB7
:1001900014308A001D2C14308A00512C14308A002F
:1001A000912C14308A00DD2C15308A001D2D15305D
:1001B0008A00512D15308A00852D15308A00B92D01
:1001C00016308A00092E16308A00172E15308A0044
:1001D000ED2D16308A00252E16308A00572E163047
:1001E0008A00312E12308A003D2AAF00C830B0009C
:1001F0000030B1000000B10BFA28B00BF828AF0BAB
:10020000F62808008316031704308C0083160313A6
:100210008301203084008001840A841F0B29A030D0
:1002200084008001840F112983171030840080011D
:10023000840A841F1729903084008001840F1D29AF
:100240008313FF30BC00FF30BD0083160130B000C7
:10025000B100B200B300B400B50083128312F130D4
:1002600086008316F13086008312E73087008316FC
:10027000FF3087008312003088008316003088002A
:100280008312C1309F0083125C201230B3004F30C4
:10029000B4005F201030B3003530B4005F2012305E
:1002A000B3005130B4005F201130B300CD30B40042
:1002B0005F2083120A30F5208312A230A0000030A4
:1002C000A1003E208316220883128039803A031D44
:1002D000892983160030A0001130A1000030A2004F
:1002E0000030A3001230A4000130A500A600A70032
:1002F000A800A900AA00AB00AC008330AD0002301A
:10030000AE000130AF008312A230A0000030A10087
:1003100044208312A230A0000E30A1000230A400BD
:100320004720A230A0000F30A1000130A4004720D8
:10033000A230A0000030A1003E20831601302E1C08
:100340000030C0000130AE1F0030C2002F08C100D5
:1003500083121230B3003D30B4005F201230B3007E
:100360005130B4005F20DC01A201A301BA29B829F1
:10037000B92908008312071AD0290708AA002A12EF
:10038000AA112A088700831607168715B7210712B6
:10039000B7218711B7218715B7210716B721BA29C9
:1003A000A030A00011224019E0293F140130DC00E8
:1003B00083160030C900FF30CA00FF30CB00831223
:1003C000A230A00011224019F029BF140230DC0035
:1003D00083160130C900FF30CA00FF30CB00831202
:1003E000A430A00011224019002A3F150330DC0080
:1003F00083160230C900FF30CA00FF30CB008312E1
:10040000A630A00011224019102ABF150430DC00CC
:1004100083160330C900FF30CA00FF30CB008312BF
:10042000212A322029181A2A1230B300F030B400E1
:100430005F20080040151230B300F230B4005F2096
:10044000080040118312C93084000008CB00840AE0
:100450000008CC00840A0008CD000310CB0CCC0CA3
:10046000CD0CCD0F362ACC0F362ACB0A18308A0095
:10047000F52000308A00CC30840048088000840ACF
:1004800049088000840A4A08800083121E30F52043
:10049000830100008317031790308D008400031739
:1004A00083168C130C1483120C088000840A8D0AA6
:1004B000F0300D06031D4F2A830183168030810022
:1004C0008312FF308F00FE308E00033090008316C1
:1004D00024309800403099008312903098001A0818
:1004E0008C1A6F2A831601308C00831200308C0026
:1004F000D0308B00DA2A8312AE142E1CAE102C20C2
:1005000003302E05023A03195C20831218198D2A34
:1005100098188D2A8C1A9A2A9D2A1812831624302C
:100520009800093099008312903098001A088C1AAC
:10053000962A9D2A18308A002829000018308A003F
:10054000EF2B0000C308031D042B2F20B60803194E
:10055000042BBE013608C207B601C21FB12AC20170
:10056000B72A17304202031CB72A1630C200BA223B
:10057000C500D92A02308A00C230420703188A0A0D
:100580004208820700340034003400340034003460
:1005900001340134023402340134003400340034B4
:1005A00000340034003400340034003401340034AA
:1005B000003400001230B3004F30B4005F20103020
:1005C000B3003530B4004208F1000319ED2A1130B0
:1005D000B4070318B30AF10BE72A00005F201230BA
:1005E000B3005130B4005F201030B3003530B40098
:1005F000420AF1000319022B1130B4070318B30AA1
:10060000F10BFC2A00005F20BB0A3B033B060839C4
:100610000319D52BBC0D3C14861E3C10BD0D3D149A
:10062000061E3D103C08803A031D1C2BFF30BE0007
:10063000C303C31BC3012A2B3D08803A031DD52BDE
:100640000130BE00C30A450A4302031C2A2B450899
:10065000C3002A2B03308A003230420703188A0A6B
:1006600042088207492B4A2B4B2B4C2B4D2B4E2BF0
:10067000AF2BAE2B4F2B722B952BB02BB12BB22B5C
:10068000B32BB42BB52BB62BB72BB82BB92BD22B46
:10069000D32BD42BD42BD42BD42BD42BD42BAE3084
:1006A0008400801BC3014308003A0319602B4308F0
:1006B000013A0319662B4308023A03196C2BD42B19
:1006C0001230B300A330B4005F20D42B1230B3003B
:1006D000AA30B4005F20D42B1230B300B130B40084
:1006E0005F20D42BAE308400801BC3014308003A46
:1006F0000319832B4308013A0319892B4308023A53
:1007000003198F2BD42B1230B300B830B4005F2004
:10071000D42B1230B300BF30B4005F20D42B123082
:10072000B300C630B4005F20D42BAE308400801BF1
:10073000C3014308003A0319A22B4308013A0319E5
:10074000A82BD42B1230B300DC30B4005F20D42BA4
:100750001230B300D730B4005F20D42BD42BD42B6D
:10076000D42BD42BD42BD42BD42BD42BD42BD42B91
:10077000D42BAE308400801BC3014308003A031918
:10078000C62B4308013A0319CC2BD42B1230B300EB
:10079000D230B4005F20D42B1230B300CD30B4007F
:1007A0005F20D42BD42BD42B00000000C308031DE2
:1007B000ED2B831622087F39B20023087F39B10060
:1007C00024083F39B00025087F39B40027081F39B5
:1007D000B3002808B500B601B701831203308A00C0
:1007E000F630420703188A0A420882070D2C102CA3
:1007F0001D2C322C472C5C2C682CAF2CF22C902D0D
:10080000F62D2A2E4B2E6C2E982EC42EE52E062F5A
:10081000272F482F6F2F8F2FA02F0000AD20B62F2E
:10082000000062200130AB004330840065200230BC
:10083000AB004C3084006520B62F0130AB00033094
:10084000840065200230AB000C308400652003304A
:10085000AB004330840065200430AB004C30840092
:100860006520B62F0330AB000330840065200430D0
:10087000AB000C30840065200530AB0043308400B1
:1008800065200630AB004C3084006520B62F053063
:10089000AB000330840065200630AB000C308400D0
:1008A00065200730AB004330840065200830AB0082
:1008B0004C3084006520B62F0730AB000330840035
:1008C00065200830AB000C3084006520C520B62FB1
:1008D000AE308400801BA72C01304306031DA72CDB
:1008E00083160030A0001130A1000030A2000030BB
:1008F000A3001230A4000130A500A600A700A800A4
:10090000A900AA00AB00AC008330AD000230AE00FD
:100910000130AF008312A230A0000030A1004420BB
:1009200000000B08F1008B138B1B932C3E20F11B56
:100930008B17831601302E1C0030C0000130AE1F13
:100940000030C2002F08C1000130B70083127D20A3
:10095000C30183120030B7008316C220B62FAE3019
:100960008400801BE82C01304306031DE82C831211
:10097000A230A0000030A1002030A4004720831640
:1009800022088312293C0318CE2C8316230A8312D3
:10099000A400A230A0000330A1004720A230A00094
:1009A0000230A1000030A4004720A230A000003097
:1009B000A1000030A40047200B08F1008B138B1B13
:1009C000DE2C3E20F11B8B1783160130B6008312FC
:1009D0007A20C30183120030B6008316B920BC20F0
:1009E000BF20B62F01304306031D232D2F20B6084C
:1009F0000319232D831630088312CA00C901C801C8
:100A000026203608CD07B60101304D0203180B2D04
:100A10001730CD00122D18304D02031C122D00305E
:100A2000CD00122DCC0129208A014A088316B0007E
:100A30008312A230A0000430A10083163008A40065
:100A40008312A4004720712002304306031D362D77
:100A50008316A01A362D8312A230A0000030A10008
:100A600083162030A0008312A40047208312003098
:100A70004306031D492D8316A01E492D8312A23063
:100A8000A0000030A10083160030A0008312A40053
:100A90004720831202304306031D7B2D2F20B6080A
:100AA00003197B2D831631088312CA00C901C801BE
:100AB00026203608CD07B60101304D020318632DFC
:100AC0003B30CD006A2D3C304D02031C6A2D0030B6
:100AD000CD006A2DCC0129208A014A088316B10075
:100AE0008312A230A0000330A10083163108A300B6
:100AF0008312A4004720742002304306031D8C2D6E
:100B00008312A230A0000230A10083160030B20090
:100B1000A2008312A40047207720B320B620B62F6E
:100B200001304306031DC12D2F20B6080319C12D26
:100B3000831633088312CA00C901C801262036086B
:100B4000CD07B60101304D020318A92D0C30CD00A0
:100B5000B02D0D304D02031CB02D0130CD00B02D55
:100B6000CC0129208A014A088316B3008312A230DF
:100B7000A0000730A10083163308A7008312A40049
:100B800047206B2002304306031DF32D2F20B608AB
:100B90000319F32D831634088312CA00C901C80152
:100BA00026203608CD07B60101304D020318DB2D93
:100BB0001F30CD00E22D20304D02031CE22D01300C
:100BC000CD00E22DCC0129208A014A088316B40009
:100BD0008312A230A0000530A10083163408A500BE
:100BE0008312A40047206E20B020B62F01304306A8
:100BF000031D272E2F20B6080319272E831635082C
:100C00008312CA00C901C80126203608CD07B601E3
:100C100001304D0203180F2E6330CD00162E6430C4
:100C20004D02031C162E0030CD00162ECC012920BB
:100C30008A014A088316B5008312A230A00008304A
:100C4000A10083163508A8008312A400472068205D
:100C5000C820B62FAE308400801B482EBE08031972
:100C6000482EB83084003E088007BE01801F3A2E0F
:100C70008001402E02300002031C402E0130800013
:100C800083168030BB188130BA1888309F008312D9
:100C90008020CB20B62FAE308400801B692EBE088A
:100CA0000319692EB93084003E088007BE01801FF9
:100CB0005B2E8001612E02300002031C612E013088
:100CC000800083168030BB188130BA1888309F00AE
:100CD00083128320CE20B62FAE308400801B942E4A
:100CE000BE080319942EBA3084003E088007BE0166
:100CF000801F7C2E8001822E03300002031C822E76
:100D000002308000831602303A06031D8D2E023019
:100D10003B0603198D2E0130BA0083168030BB18B4
:100D20008130BA1888309F0083128620D120B62FD8
:100D3000AE308400801BC02EBE080319C02EBB300D
:100D400084003E088007BE01801FA82E8001AE2EC1
:100D500003300002031CAE2E0230800083160230E6
:100D60003B060319B92E02303A06031DB92E023094
:100D7000BB0083168030BB188130BA1888309F00C2
:100D800083128920D420B62FAE308400801BE22E3F
:100D9000BE080319E22EBC3084003E088007BE0165
:100DA000801FD42E8001DA2E02300002031CDA2EBE
:100DB0000130800083168030BB188130BA1888302B
:100DC0009F0083128C20D720B62FAE308400801B6A
:100DD000032FBE080319032FBD3084003E0880078F
:100DE000BE01801FF52E8001FB2E02300002031C85
:100DF000FB2E0130800083168030BB188130BA187A
:100E000088309F0083128F20DA20B62FAE30840006
:100E1000801B242FBE080319242FBE3084003E08F7
:100E20008007BE01801F162F80011C2F0230000298
:100E3000031C1C2F0130800083168030BB188130CA
:100E4000BA1888309F0083129220DD20B62FAE3072
:100E50008400801B452FBE080319452FBF30840036
:100E60003E088007BE01801F372F80013D2F0230D2
:100E70000002031C3D2F0130800083168030BB1818
:100E80008130BA1888309F0083129520E620B62F53
:100E9000AE308400801B6B2FBE0803196B2FC0304F
:100EA00084003E088007BE01801F582F80015E2FFE
:100EB00002300002031C5E2F013080008312A2303A
:100EC000A0000E30A10083160330401C0230AE009B
:100ED0008312A40047209E20E020E320B62F01309B
:100EE0004306031D8B2FAE308400801B8B2F2F20D9
:100EF000B60803198B2FC130840036088007B6016D
:100F00008312A230A0000F30A10083164108AF0069
:100F10008312A400472098209B20E920B62FAE30F2
:100F20008400801B9C2FBE0803199C2F01303E06B5
:100F3000031D9C2FBE01C015A120EC20EF20B62F71
:100F4000BE080319B12FC230840001303E06031DD4
:100F5000AB2FC014B12FFF303E06031DB12F40143C
:100F6000B12F8301BE01A420A720B62F00007B2A49
:101000000000CC0148080F39CD0003104D0DCF0072
:101010004C0DCE000310CD0DCC0D0310CD0DCC0D1D
:101020000310CD0DCC0D4F08CD070318CC0A4E0888
:10103000CC07490E0F39CD070318CC0A03104D0D0C
:10104000CF004C0DCE000310CD0DCC0D0310CD0DF7
:10105000CC0D0310CD0DCC0D4F08CD070318CC0AD5
:101060004E08CC0749080F39CD070318CC0A0310E6
:101070004D0DCF004C0DCE000310CD0DCC0D031047
:10108000CD0DCC0D0310CD0DCC0D4F08CD070318A1
:10109000CC0A4E08CC074A0E0F39CD070318CC0AEC
:1010A00003104D0DCF004C0DCE000310CD0DCC0D17
:1010B0000310CD0DCC0D0310CD0DCC0D4F08CD0779
:1010C0000318CC0A4E08CC074A080F39CD0703187D
:1010D000CC0A8A010800B50CB50C3030B5050608FD
:1010E000C039B50408308A00350EB7007C303707A8
:1010F00003188A0A37088207922892289228922891
:10110000922892289228922892289228922892280F
:1011100092288F288C2892280130B6079328FF3018
:10112000B607932800008A0108000B08EE008B1315
:101130008B1B972800007A22A91020102008282253
:1011400029182A29A9102108282229182A29A91092
:101150002914831620088312203900382822A91068
:1011600029148316210883121F3900382822A91058
:101170002914831622088312003900382822A91066
:1011800029148316230883127F3900382822A910D6
:1011900029148316240883123F3900382822A91005
:1011A00029148316250883123F3900382822A910F4
:1011B0002914831626088312073900382822A9101B
:1011C00029148316270883121F3900382822A910F2
:1011D0002914831628088312FF3900382822A91001
:1011E0002914831629088312FF3900382822A910F0
:1011F000291483162A088312FF3900382822A910DF
:10120000291483162B088312FF3900382822A910CD
:10121000291483162C088312FF3900382822A910BC
:10122000291483162D088312833900382822A91027
:10123000291483162E088312833900382822A91016
:10124000291483162F08831228229222EE1B8B1753
:101250008A0108009222EE1B8B178A0108000B08F6
:10126000EF008B138B1B312900007A22A91020106C
:101270002008282229184A29A910210828222918DB
:101280004A29A9102914240828229222EF1B8B171F
:101290008A0108009222EF1B8B178A0108000B08B5
:1012A000EC008B138B1B512900007A22A91020100F
:1012B000200828222918F829A910210828222918ED
:1012C000F8297A22A9102014200828222918F829A0
:1012D000A9142910FF30282226088316A0008312A3
:1012E000A9142910FF30282226088316BF39A1002F
:1012F0008312A9142910FF30282226088316A20081
:101300008312A9142910FF302822260883167F395A
:10131000A3008312A9142910FF302822260883165F
:101320003F39A4008312A9142910FF30282226086F
:1013300083163F39A5008312A9142910FF302822F3
:10134000260883160739A6008312A9142910FF3036
:101350002822260883169F39A7008312A914291072
:10136000FF30282226088316A8008312A91429100A
:10137000FF30282226088316A9008312A9142910F9
:10138000FF30282226088316BF39AA008312A91429
:101390002910FF30282226088316BF39AB0083129C
:1013A000A9142910FF302822260883168739AC009B
:1013B0008312A9142910FF302822260883168339A6
:1013C000AD008312A9142910FF30282226088316A5
:1013D0008339AE008312A9142914FF30282226086D
:1013E0008316AF0083129222EC1B8B178A01080030
:1013F0009222EC1B8B178A0108000B08ED008B135F
:101400008B1BFF297A22A9102010200828222918D6
:10141000232AA910210828222918232A7A22A91070
:101420002014200828222918232AA9142914FF305F
:101430002822A03021078400260880009222ED1B7C
:101440008B178A0108009222ED1B8B178A01080076
:10145000A500A6010830A800A50D83160715031CDA
:1014600007118312A723831687148312A723A60DBF
:101470002614071D2610831687108312A80B2C2A0A
:10148000831607158312A723A918632A83168714C6
:101490008312A7236430A800071D592AA80B4C2AE1
:1014A0002914831687108312A7238316071183122A
:1014B00008002910831687108312A72383160711AB
:1014C0008312A7230800291C692A83160715831293
:1014D0006C2A831607118312A7238316871483129D
:1014E000A723831687108312A7238316071183125D
:1014F000A723080083120708AA002A11AA102A08A5
:101500008700831607158312A72383168714831277
:10151000A723831607118312A7238316871083122C
:10152000A7230800A723831687148312A7238316F3
:1015300007158312A72308000B08E8008B138B1BE9
:101540009E2A6430F30029117823A9102010200866
:1015500022232918B12A94232911E81B8B178A0109
:1015600008009423F30BA32A2915E81B8B178A0183
:1015700008000B08EA008B138B1BBB2AF301000049
:101580007823A910201020082223291CCF2A942375
:10159000F30BC02A2915EA1B8B178A010800A91032
:1015A000220822232918EC2AA9102308222329180B
:1015B000EC2A7823A9102014200822232918EC2AC9
:1015C000A9142914FF3022232608A40094232911EA
:1015D000EA1B8B178A01080094232915EA1B8B1735
:1015E0008A0108000B08EB008B138B1BF42AF30114
:1015F00000007823A910201020082223291C082B82
:101600009423F30BF82A2915EB1B8B178A0108008A
:10161000A9102208222329181C2BA91023082223F1
:1016200029181C2BA91029142408222394232911DA
:10163000EB1B8B178A01080094232915EB1B8B17D2
:101640008A010800A500A6010830A800A50D831690
:101650000716031C07128312A723A72383168715D7
:101660008312A723A60D2614071E261083168711A2
:101670008312A723A80B262B831607168312A723F2
:10168000A918612B831687158312A723C830A800D9
:10169000071E552BA80B482B29148316871183127C
:1016A000A7238316071283120800291083168711B7
:1016B0008312A723831607128312A723A723A72326
:1016C0000800291C672B8316071683126A2B8316C2
:1016D00007128312A723831687158312A723831665
:1016E00087118312A723831607128312A7230800EA
:1016F00083120708AA002A12AA112A088700831653
:1017000007168312A723A723831687158312A723FF
:10171000A723831607128312A723A72383168711F3
:101720008312A723A7230800A723831687118312F8
:10173000A723831607128312A723A72383168715CF
:101740008312A723831607168312A7230800080015
:10200000000083120608AD002D11AD10AD112D0892
:102010008600B827000074267426742692268A014A
:102020000800831233088A003530B40234083420A3
:10203000AC00AC1F2B282C08FE3A031D212880265B
:102040002C282C08FF3A031D27288A010800AC130E
:102050002C08AA262C280227B40A35303407031985
:10206000B30A33088A001628820738346334683488
:1020700020343134303462346934743420344C3494
:102080004F344734473445345234FF3420345634C7
:102090006534723431342E343034323420342034C8
:1020A00028344D3465346D342D342934FF344334B1
:1020B0003034203420342034203420342034203470
:1020C0004334313420342034203420342034FF345D
:1020D0004334323420342D342D342D342D342034F7
:1020E00020344334333420342D342D342D342D34E6
:1020F000FF344334343420342D342D342D342D34F6
:10210000203420344334353420342D342D342D34D0
:102110002D34FF344334363420342D342D342D34D3
:102120002D34203420344334373420342D342D34AE
:102130002D342D34FF34523454344334203472342B
:1021400065347334653474342034203420342034BE
:10215000203420342034FF34543469346D346534F1
:1021600020347A34653472346F342034203420348F
:102170002034203420342034FF34543469346D3416
:1021800065342034203420342D342D343A342D3429
:102190002D343A342D342D342034FF34443461341A
:1021A00074346534203420342034203420342034F6
:1021B0002D342D342F342D342D342034FF34593424
:1021C0006534613472342034203420342034203497
:1021D000203420342D342D342D342D342034FF344C
:1021E00043344834303420346D346F3464346534CF
:1021F00020342034203420342D342D342D34203418
:10220000FF3443344834313420346D346F34643413
:10221000653420342034203420342D342D342D34B2
:102220002034FF3443344834323420346D346F3436
:102230006434653428342D34293420342D342D343D
:102240002D342034FF3443344834333420346D3457
:102250006F346434653428342B34293420342D34DD
:102260002D342D342034FF34433448343434203476
:102270006D346F3464346534203420342034203499
:102280002D342D342D342034FF3443344834353448
:1022900020346D346F346434653420342034203479
:1022A00020342D342D342D342034FF34433448343D
:1022B000363420346D346F34643465342034203443
:1022C000203420342D342D342D342034FF34433445
:1022D0004834373420346D346F34643465342034FA
:1022E0002034203420342D342D342D342034FF3448
:1022F00050346534723469346F34643455346E3418
:1023000069347434203420342D342D342D34203469
:10231000FF3450346534723469346F346434283493
:102320002D342D342D3429342034203420342034DD
:102330002034FF34413464342D342D342D342D3485
:102340002D342D342F342D342D342D342D342D3483
:102350002D342034FF344C344F3447342E342D3454
:102360002D342034203420342034203420342D34B3
:102370002D342D342034FF342034203420342034C4
:1023800020342034203420342034203420342034AD
:102390002034203420342034FF34203469346E3427
:1023A00069347434693461346C3469347A3469342E
:1023B0006E3467342E342E342E34FF342A342034D5
:1023C000413444342034433448342E34203461348E
:1023D0006C346C3420346F3466346634FF342A3401
:1023E0002034443469347234653463347434723460
:1023F000793420346F347634653472342034FF34C9
:102400002A3420344134643464347234653473348F
:10241000733420346F34763465347234203420348D
:10242000FF344634693472346D3477346134723435
:102430006534203455347034643461347434653414
:102440002034FF348F342A34FF348F342034FF3467
:102450008F347834FF3480342034203420342034D6
:1024600020342034203420342034203420342034CC
:102470002034203420342034FF34C034203420343D
:1024800020342034203420342034203420342034AC
:10249000203420342034203420342034FF3480345D
:1024A000FF34C034FF348C3420346F346E34FF3446
:1024B000CC3420346F346E34FF348C346F34663453
:1024C0006634FF34CC346F3466346634FF348C3475
:1024D000763466342D34FF34CC34763466342D347F
:1024E000FF348C34763466342B34FF34CC34763479
:1024F00066342B34FF348C34733465346334FF34E6
:10250000CC34733465346334FF348C346D346934C3
:102510006E34FF34CC346D3469346E34FF348C3413
:10252000203420342034FF34CC3420342034203480
:10253000FF348C3420346F346B34FF34CC3420348B
:102540006F346B34FF348634203489343A348C341D
:102550003A34FF3486345B3489345D348C343A3415
:10256000FF348634203489345B348C345D34FF345A
:10257000893420348C342F348F342034FF34893420
:102580005B348C345D348F342034FF348934203410
:102590008C345B348F345D34FF348B345B348F3454
:1025A0005D34FF348B3420348F342034FF348A344C
:1025B0005B348F345D34FF348A3420348F342034DC
:1025C000FF342D342D342D342D34FF34563446341D
:1025D00020342D34FF345634463420342B34FF3429
:1025E0006F34FF345F34FF340E30F72A4E30AA26A2
:1025F0005C080F39303801278A0108000408AA2630
:10260000B7302B078400003000060319102B01306F
:1026100000060319182B023000060319282B412B42
:102620001230B300E130B400112013308A00412B86
:10263000CF302B0784000008CC00D7302B07840054
:102640000008CD002A274930612713308A00412B2A
:1026500003302B060319312B04302B060319392BB9
:10266000412B1230B300E630B400112013308A0041
:10267000412B1230B300EB30B400112013308A002C
:10268000412B8A0108000730462B4730AA268316C3
:10269000300E83120F393038012783163008831229
:1026A0000F39303801278A0108000A30582B4A3088
:1026B000AA268316310E83120F393038012783166C
:1026C000310883120F39303801278A0108000D3094
:1026D0006A2B4D30AA268316320E83120739303802
:1026E00001278316320883120F39303801278A01F7
:1026F00008000A307C2B4A30AA268316330E831238
:102700000739303801278316330883120F393038E0
:1027100001278A0108000D308E2B4D30AA26831622
:10272000340E83120F393038012783163408831290
:102730000F39303801278A0108000B30A02B4B30AD
:10274000AA2632300127303001278316350E831236
:102750000F39303801278316350883120F39303886
:1027600001278A0108000130831636068312031DF3
:10277000BF2B1230B3009930B400112008008A0139
:1027800008000030831636068312031DCD2B12304D
:10279000B3009430B40011200800013083163606CF
:1027A0008312031DD92B1230B3009430B4001120D2
:1027B00008008A0108000130831637068312031DC2
:1027C000E72B1230B3009930B400112008008A01C1
:1027D00008000030831637068312031DF52B1230D4
:1027E000B3009430B400112008000130831637067E
:1027F0008312031D012C1230B3009430B400112059
:1028000008008A0108000030831638068312031D71
:102810000F2C1230B3005D30B400112008000130DD
:10282000831638068312031D1B2C1230B30053305D
:10283000B400112008008A01080000308316380611
:102840008312031D292C1230B3006230B400112012
:1028500008000130831638068312031D352C123010
:10286000B3005830B400112008008A01080000307D
:10287000831639068312031D432C1230B3005D30DA
:10288000B400112008000130831639068312031D9D
:102890004F2C1230B3005330B400112008008A01CD
:1028A00008000030831639068312031D5D2C123098
:1028B000B3006230B40011200800013083163906DD
:1028C0008312031D692C1230B3005830B40011205C
:1028D00008008A010800003083163A068312031D9F
:1028E000772C1230B3005D30B400112008000130A5
:1028F00083163A068312031D832C1230B300533023
:10290000B40011200800023083163A068312031D1A
:102910008F2C1230B3006730B400112008008A01F8
:102920000800003083163A068312031D9D2C1230D6
:10293000B3006230B40011200800013083163A065B
:102940008312031DA92C1230B3005830B40011209B
:102950000800023083163A068312031DB52C12308C
:10296000B3006C30B400112008008A010800003068
:1029700083163B068312031DC32C1230B3005D3057
:10298000B40011200800013083163B068312031D9A
:10299000CF2C1230B3005330B400112008000230A5
:1029A00083163B068312031DDB2C1230B3007130FB
:1029B000B400112008008A010800003083163B068D
:1029C0008312031DE92C1230B3006230B4001120D1
:1029D0000800013083163B068312031DF52C1230CC
:1029E000B3005830B40011200800023083163B06B3
:1029F0008312031D012D1230B3007630B400112074
:102A000008008A010800003083163C068312031D6B
:102A10000F2D1230B3005D30B400112008000130DA
:102A200083163C068312031D1B2D1230B300533056
:102A3000B400112008008A010800003083163C060B
:102A40008312031D292D1230B3006230B40011200F
:102A50000800013083163C068312031D352D123009
:102A6000B3005830B400112008008A01080000307B
:102A700083163D068312031D432D1230B3005D30D3
:102A8000B40011200800013083163D068312031D97
:102A90004F2D1230B3005330B400112008008A01CA
:102AA0000800003083163D068312031D5D2D123091
:102AB000B3006230B40011200800013083163D06D7
:102AC0008312031D692D1230B3005830B400112059
:102AD00008008A010800003083163E068312031D99
:102AE000772D1230B3005D30B400112008000130A2
:102AF00083163E068312031D832D1230B30053301C
:102B0000B400112008008A010800003083163E0638
:102B10008312031D912D1230B3006230B4001120D6
:102B20000800013083163E068312031D9D2D1230CE
:102B3000B3005830B400112008008A0108000030AA
:102B400083163F068312031DAB2D1230B3005D3098
:102B5000B40011200800013083163F068312031DC4
:102B6000B72D1230B3005330B400112008008A0191
:102B70000800003083163F068312031DC52D123056
:102B8000B3006230B40011200800013083163F0604
:102B90008312031DD12D1230B3005830B400112020
:102BA00008008A0108000030831640068312031DC6
:102BB000DF2D1230B3007B30B4001120080001304B
:102BC000831640068312031DEB2D1230B3008530AF
:102BD000B400112008008A01080000308316400666
:102BE0008312031DF92D1230B3008030B400112080
:102BF00008000130831640068312031D052E123093
:102C0000B3008A30B400112008008A0108000730A0
:102C10000A2E4730AA26CC0183162F088312CD0036
:102C20002A27493064278A0108000C30182E4C30BE
:102C3000AA26CC01831641088312CD002A274930E9
:102C400064278A0108000230262E4230AA26C630A8
:102C50005B272F300127CC305B278A010800043026
:102C6000322E4430AA26CC0183164F088312CD00A1
:102C70002A274A3067278A01080000308316420657
:102C80008312031D492E1230B3005D30B4001120B1
:102C900008000130831642068312031D552E1230A0
:102CA000B3005330B400112008008A01080000303E
:102CB000831642068312031D632E1230B300623066
:102CC000B400112008000130831642068312031D50
:102CD0006F2E1230B3005830B400112008008A0162
:102CE000080001278A01080083123830AC00FE2654
:102CF000B827080083122030AC00FE26B827080051
:102D000083120130AC00B026FE2608008312023088
:102D1000AC00B026FE26080083120630AC00B026B8
:102D2000FE26080083120C30AC00B026FE260800F8
:102D300083120D30AC00B026FE26080083121C3032
:102D4000AC00B026FE26080083124038AC00B02646
:102D5000FE26080083128038AC00B026FE2608004C
:102D60008316FF30880083126430B2000611861487
:102D7000B92EBA2EBB2EBC2EBD2EBE2EBF2EC02EFF
:102D80008615C22EC32EC42EC52EC62EC72EC82E03
:102D9000C92E0808AD008611AD1FD12EB20BB62E7C
:102DA0000000831600308800831208008316FF306D
:102DB000880083122E106430B20006118614E02EB3
:102DC000E12EE22EE32EE42EE52EE62EE72E8615EA
:102DD000E92EEA2EEB2EEC2EED2EEE2EEF2EF02E1F
:102DE0000808AD008611AD1FF82EB20BDD2E2E1493
:102DF00083160030880083128A01080006118610AD
:102E00000B2FAC00B026061586100B2FAC000B273D
:102E1000AC0E0B2708002C0888000814AC1C081006
:102E200088142C1C8810142F152F162F172F182FCD
:102E3000192F1A2F1B2F86151D2F1E2F1F2F202FE6
:102E4000212F222F232F242F861108000030CC00A1
:102E50006430CD000F30F400C801C901CA0103106D
:102E6000CD0DCC0DCA0DC90DC80D03304A07F300B6
:102E7000F319CA0030304A07F300F31BCA000330CD
:102E80004907F300F319C90030304907F300F31B79
:102E9000C90003304807F300F319C8003030480771
:102EA000F300F31BC800F40B302FCD0DCC0DCA0D71
:102EB000C90DC80D08008400F3016A2F8400F301D6
:102EC000772F8400F301852F8400F301922F840073
:102ED000F301A02F7318722F000E0F39031D722FEC
:102EE0002030762F7314000E0F39303801277318F5
:102EF0007F2F00080F39031D7F2F2030832F73147D
:102F000000080F3930380127840A73188D2F000EFE
:102F10000F39031D8D2F2030912F7314000E0F39A0
:102F20003038012773189A2F00080F39031D9A2F84
:102F300020309E2F731400080F3930380127840A7F
:102F40007318A82F000E0F39031DA82F2030AC2FA7
:102F50007314000E0F393038012700080F3930384C
:102F6000012708000130CA2F0230CA2F0A30CA2FA9
:102F70002830CA2FC830CA2FBA27BA270800BA2764
:102F8000BA27BA27BA2708000A30B100BA27B10B0E
:102F9000C62F08008312AF00B0010000B00BCD2F88
:062FA000AF0BCC2F08006E
:10300000000083124018C22883160C178312F501A2
:10301000B8307507840001300006031DBC28D201BA
:10302000D1017508F600F60DF60D760D3839F6006B
:10303000C7301F0576049F001030D0004D30F600D9
:10304000F60B20280C1347308B051F1583160C1028
:103050008312F8308B05630000001F192D2883169A
:103060000C14831250308B0483161E088312D2076F
:103070000318D10A1E08D107D00B1E280430D00037
:10308000D10CD20CD00B40280F30D105D8307507A9
:10309000840052088000D0307507840051088000F9
:1030A0005208F6001F39D200F60DD10DF60DD10DE4
:1030B000F60DD10D1F30D105750EF600760DE039F5
:1030C000D104D2048316430D83120E39A038D300E5
:1030D000831644088312D400831645088312D50052
:1030E0005308A0005408A2005508A3005108A400EA
:1030F00008308A00F22218308A008316C50F832810
:10310000C40F8328C30A83128316430D83120E391A
:10311000A038D300831644088312D40083164508D0
:103120008312D5005308A0005408A2005508A3003C
:103130005208A40008308A00F22218308A00831650
:1031400049084306031DB6284A084406031DB6284D
:103150004B084506031DB6288316C50FB228C40FB9
:10316000B228C30A831240144016C2288316C50F22
:10317000BC28C40FBC28C30A8312F50A08307506A0
:10318000031D08288312C33084000008CB00840A82
:103190000008CC00840A0008CD000310CB0CCC0C36
:1031A000CD0CF520C630840048088000840A490808
:1031B0008000840A4A08800083160C1383128A0157
:1031C0001B28FF308F00FF308E008312A230A0003A
:1031D0000030A10009308A004F218A0113280030F5
:1031E000CB000030CC006430CD001730F400C801B3
:1031F000C901CA010310CD0DCC0DCB0DCA0DC90DEF
:10320000C80D03304A07F300F319CA0030304A07EB
:10321000F300F31BCA0003304907F300F319C90098
:1032200030304907F300F31BC90003304807F300AF
:10323000F319C80030304807F300F31BC800F40B43
:10324000FB28CD0DCC0DCB0DCA0DC90DC80D080046
:10325000830118080639003A0319322918121A088E
:103260001816DB2B1A08D700FF30570603193D2923
:103270000030570603193D294F2999308400000872
:10328000403A031D44294729403080004A2915301F
:1032900080004A290C1E4A29FC309900DB2B0000D3
:1032A000FC305706031D59290C1E5429FC30990087
:1032B000DB2B00003F305706031D65298316981C41
:1032C0005F2983123F309900DB2B00004630570600
:1032D000031D9329831203131230B3004F30B4003F
:1032E00010308A00112018308A001230B3001130DB
:1032F000B40010308A00112018308A0083120313A2
:103300001230B3005130B40010308A001120183050
:103310008A001130B300BC30B40010308A00112094
:1033200018308A00002F56305706031DE0298316F7
:10333000981C982983124C3099008316981C9E295A
:1033400083124F3099008316981CA42983124730AA
:1033500099008316981CAA29831247309900831676
:10336000981CB0298312453099008316981CB62901
:103370008312523099008316981CBC298312203086
:1033800099008316981CC22983125630990083161F
:10339000981CC8298312313099008316981CCE29B5
:1033A00083122E3099008316981CD4298312303052
:1033B00099008316981CDA29831232309900DB2B8E
:1033C000000053305706031DE729C014DB2B000013
:1033D00045305706031DEE294014DB2B00008316F1
:1033E0004218B72B831250305706031D332A831619
:1033F000981CF82983120D30990083128C1EFE2927
:103400001A08D7000D3A0319DB2BC0308400570887
:1034100080008C1E092A1A08D7000D3A0319DB2BED
:10342000C13084005708800008308A008312A2301F
:10343000A0000E30A10083160330401C0230AE0005
:103440008312A4002F2108308A008312A230A0002A
:103450000F30A10083164108AF008312A4002F2172
:1034600018308A00DB2B000041305706031D572A15
:103470008316981C392A83120D30990083128C1EF2
:103480003F2A1A08D7000D3A0319DB2BB830840005
:10349000570E0F3984070F30570580008316803090
:1034A000BB188130BA1888309F0083123F2A000071
:1034B00043305706031D5E2AC015DB2B00004C303D
:1034C0005706031D762A8316981C642A490883121E
:1034D00099008316981C6A2A4A0883129900831659
:1034E000981C702A4B0883129900DB2B00006C306B
:1034F0005706031D8E2A8316981C7C2A43088312C4
:1035000099008316981C822A440883129900831616
:10351000981C882A450883129900DB2B0000443050
:103520005706031DA72A8317903084008316981C22
:10353000972A831200089900840AF0300406031DBC
:10354000962A831383164F0883129900DB2B000001
:1035500052305706031D822B83121230B3002230E3
:10356000B40010308A00112018308A0083120B0832
:10357000EA008B138B1BB92A8312D901DA01DB0114
:10358000590D0E39A038A00008308A007823183071
:103590008A0008308A00A910201020082223183041
:1035A0008A00291CDE2A08308A00942318308A00F9
:1035B000F10BC02A2915EA1B8B17B72B08308A009C
:1035C000A9105A08222318308A002918B72B08306E
:1035D0008A00A9105B08222318308A002918B72B0B
:1035E00008308A00782318308A0008308A00A91031
:1035F00020142008222318308A002918B72BFF3006
:103600005B06031D0A2BFF305A06031D0A2BA91463
:1036100029140C2BA914291008308A00FF3022230A
:1036200018308A002608A4008316981C152B8312D4
:1036300024089900DB0F1F2BDA0F1F2BD90A031761
:10364000831210308D00031783160C140317831296
:103650000C08031383125906031D622B03178312F0
:1036600011308D00031783160C14031783120C08F6
:10367000031383125A06031D622B031783121230A1
:103680008D00031783160C14031783120C08031301
:1036900083125B06031D622BA914291408308A00CB
:1036A000FF30222318308A002608A4008316981CB5
:1036B000572B83122408990008308A00942318306D
:1036C0008A00732B00305B06031DFF2A00305A0668
:1036D000031DFF2A08308A00942318308A005908F5
:1036E0005C06031DC02A83122911EA1B8B17831263
:1036F0001230B3002530B40010308A001120183089
:103700008A00DB2B000072305706031D952BA0307A
:1037100084008316981C8A2B831200089900840A5F
:103720000408B03C031D892BDB2B000077305706C3
:10373000031DB62B8316981C9B2B83120D3099000A
:10374000A03084008B138B1BA22B83128C1EA62B04
:103750001A088000840A0408B03C031DA52B083019
:103760008A00952018308A008B17DB2B000083120B
:103770001230B3002830B40010308A001120183005
:103780008A0008308A00942318308A008316981C17
:10379000C72B8312453099008316981CCD2B8312BA
:1037A000523099008316981CD32B83125230990003
:1037B00000308A009D2A83121230B3002530B400F5
:1037C00010308A00112018308A008316981CE62BCE
:1037D00083120D309900831200308A009D2A000068
:1037E000C01CDE2CC01083164218DE2C8312083059
:1037F000F100BF308400013000060319162C840349
:10380000F10BFB2B83121230B3005130B400103097
:103810008A00112018308A001130B300DE30B40065
:1038200010308A00112018308A00DE2C83160630F2
:103830004F06031D2F2C83121230B3005130B400F9
:1038400010308A00112018308A001130B300EF3098
:10385000B40010308A00112018308A00DE2C831644
:1038600043084902031C352C492C83121230B30043
:103870005130B40010308A00112018308A00123004
:10388000B3000030B40010308A00112018308A00D4
:10389000DE2C8316CF0A4F088312F100840110300A
:1038A0008407F10B4F2C803084078317831635086B
:1038B0008000840A33088000840A34088000840A67
:1038C00030088000840A31088000840A32088000B1
:1038D000840A40088000840A41088000F101F20156
:1038E000F20DF10DF20DF10DFC30F2053808F20485
:1038F000F20DF10DF20DF10DFC30F2053908F20474
:10390000F20DF10DF20DF10DFC30F2053A08F20462
:10391000F20DF10DF20DF10DFC30F2053B08F20451
:10392000F20DF10DF20DF10DFC30F2053C08F20440
:10393000F20DF10DF20DF10DFC30F2053D08F2042F
:10394000F20DF10DF20DF10DFC30F2053E08F2041E
:10395000F20DF10DF20DF10DFC30F2053F08F2040D
:10396000840A71088000840A72088000831383121D
:10397000A230A0000F30A10083164108AF008312CF
:10398000A40008308A002F2118308A008312A23048
:10399000A0000E30A10083164214AE172E08831229
:1039A000A40008308A002F2118308A0083120610E4
:1039B000831606108401840BDB2C06148312401C32
:1039C0007D2D40108316421C7D2D83120B12A230D8
:1039D000A0000E30A10083164210AE132E088312F1
:1039E000A40008308A002F2118308A00C830AE00A9
:1039F000A4010000AE0BF92CA40BF92C8B100B16B4
:103A000083164F088312F100840110308407F10BF4
:103A1000052D8A3084078316831743088000840AA3
:103A200044088000840A45088000840AFF30800032
:103A3000840AFF308000840AFF3080009F308400B9
:103A40004F088000AF3084004F088000BF308400F2
:103A50004F088000CF3084004F088000DF308400A2
:103A60004F088000EF3084004F0880008B138B1BC1
:103A7000362D83010317831290308D0003178316B0
:103A80001008031783128C006E258301031783121D
:103A900010308D00031383164308031783128C0024
:103AA0006E2583010317831211308D0003138316D3
:103AB0004408031783128C006E25830103178312B9
:103AC00012308D00031383164508031783128C00F0
:103AD0006E2583018B178B1F6A2D7D2D031783168F
:103AE0008C130C1555308D00AA308D008C148C1859
:103AF000772D031783128D01080083128312C01DD6
:103B00008E2DC011831642188E2D8316CF01C3014E
:103B1000C401C501C601C701C80183128312003068
:043B20008A00A12A4C
:103E0000831603138C018D01831203138C018D0122
:103E10008B01FB01831603132430980083120313D4
:103E2000903098001A088C1A122F831603170C1161
:103E3000831203131808840006390319252F180864
:103E40000639023A0319582F5F2F8C1E152F1A08B6
:103E50008400FB1F492F1F308A007B08033982072B
:103E6000342F382F3C2F402F0408FC00FB0A152F5D
:103E70000408FD00FB0A152F0408FE00FB0A152F9D
:103E80000408FF006B270C1E432F40309900FB01F4
:103E9000152F04083F3A031D502F8527FB01152FCE
:103EA0000408413A031D572F8030FB00152F152FB2
:103EB000181218161A088C1A5A2F4F30662F18121B
:103EC00018161A088C1A612F4630662F0C1E662FA2
:103ED0009900FB01152F031783127C088F007D08C2
:103EE0008D007E088E007F088C0083168C170C15C1
:103EF0008B1355308D00AA308D008C14000000000B
:103F00008C18802F0C118301080010308400FB01F5
:103F10000C1E882FE0279900FB0A840B882F840150
:043F2000FB01080099
:103FC0001F308A007B088207413445342D344C343D
:103FD0004F34473447344534523420345634303427
:083FE00031342E343034323448
:084000000000010000000200B5
:02400E00723FFF
:00000001FF
